:10000000002A0800B70B0928AA0B09282408031D99
:100010008F2B0230831687008312002DC120012010
:10002000122DC1200130831687008312282DC12094
:1000300001203A2DC120A80B8C2CA80ABA0B262827
:10004000BA0AA51325088600071507118030360265
:1000500003193820B608031DB60B0228BA01B212E4
:100060003311A6113217A7014820251B321302288D
:1000700027088A0182074528B2298929F129BE2942
:10008000C529B529E128DE29E8283311A6114E2813
:10009000390A0739C4000030C50052282708C400B7
:1000A0000A30C500F6302302C000F6302202C1003B
:1000B000F6302102C200F6302002C3004008AD2015
:1000C000AC004108AD20AD004208AD20AE004308B1
:1000D00003190B30AD20AF004408AD20B000450837
:1000E000AD20B100B117261EB113B017A61DB01375
:1000F000250886000715071100343315A615B5012C
:10010000A703270F85283B03A7000A1527088200AD
:100110003315A615B501A70A3B0827020319A70145
:1001200027080A15820027088A018207362997299D
:100130008329F729C329D229BB29E628EA29F428EB
:1001400027088A0182075729A6297D29F429C12970
:10015000C829B829E428E129EB288A0182078134DB
:10016000E7349234C234E434C8348834E13480341F
:10017000C034FB34FF34FE34A134B83481348634C7
:100180008C348316FF30860083122830A900640067
:10019000A90BC7280F30B2040608A9000608F038DA
:1001A0000F3AB205831686018312B316051AB312ED
:1001B0003317851D3313B314851A0029B310331375
:1001C0000029251DAC29A1292511AC292515A12916
:1001D0007322390A8C29033039050319F128B90330
:1001E000E828B9143914E828033039020319FA2829
:0A01F000B90AE8280030B900E82839
:10020000240E2918AA00F030AB0529052B02031D86
:100210002029F030290503191C29B50B7C28291A3F
:100220008F2B291B502D0130B500B40B7C280030DA
:10023000AB000F30B4007C28B5010030AB007C2847
:10024000B216A517BA01C030B600240EAA000130BC
:10025000A8000F30B4002908AB002B1A7D28AB1A78
:1002600093282B1B8828AB1BA0287C283311A611B0
:10027000A30F4E28F630A300A20F4E28F630A2009E
:10028000A10F4929F630A100A00F5029F630A00097
:100290007C28F8302102031D4E28FE30A10044299D
:1002A000F8302002031D4E28F630A0004E283311EE
:1002B000A611F530A3032302031D4E28FF30A3002F
:1002C000F530A2032202031D4E28FF30A200F530B4
:1002D000A1032102031D7629FF30A100F530A00300
:1002E0002002031D4E28F730A0004E28FD302102C9
:1002F000031D4E28F730A1006E29A403240F89297D
:100300000930A4008929A40A0A3024020319A4018F
:10031000892924080319AC29C000C1010B30C2008F
:100320000B30C3002708C4000A30C5005E28A5149E
:100330002508860007150711A901B311A90B9E29ED
:10034000002B0F30C1000D30C0008E29A5102508EC
:10035000860007150711B3150F30C2000E30C1001B
:10036000C0009029A51CAC29A129251FAC29A129D1
:1003700032172513AC2932132517A1292518AC29CA
:10038000A1292510AC292514A129A51EC929D329E5
:10039000A5120C30C3000930C2001030C10011306A
:1003A000C0009229A5160B30C3000030C200CD2931
:1003B000A511BC18A51525123C1C251607303C05B7
:1003C000A62A07303C050319E729BC03D8293C15A8
:1003D000BC03D829BC0A3C19EE29D829F830BC0541
:1003E000D829261FAC29A12933162613AC2933128C
:0403F0002617A12902
:1004000085018701860183160030860087008312EC
:1004100007150711FF308600071607128716871287
:100420000717071387178713B7018B018316F83057
:100430008500FF308600003087008C308100063058
:100440009F0083120A30BB00A901B801A9176400FC
:10045000A80B272A8715061F2F2AA90B272A000079
:10046000FE30AC00AD00AE00AF00B000B100FF3018
:10047000B200B30000308500CA00AB01A800C03054
:10048000B60035305830A600A7013F309C22033912
:10049000B9006400061B652A7322240EAA00A70176
:1004A000831686018312A510A517BA0125088600B8
:1004B000071507113316261B3312BC01BC10A519F2
:1004C000BC143C10251E3C140228FB30A300FD3058
:1004D000A200FE30A100F630A0000230A400583087
:1004E000A600A5014D2AB90E39089C22A0000130B2
:1004F00039079C22A100023039079C22A200033058
:1005000039079C22A300043039079C22A40005303F
:1005100039079C22A9008230A5057D302905A50454
:10052000063039079C22A9002613291B26170730FD
:1005300039079C22B90E0800031783128D00831619
:100540008C130C1483120C08031308000339A90040
:100550008A018A14E330AC008130AD00BD30AE00BA
:100560009D30AF000310A90D0310A90D0310290D34
:1005700082070000A030AD009D30AE00B830AF0063
:10058000D72A0530AC0000009D30AE00FF30AF0030
:10059000D72AA430AC008830AD000000A430AF00F2
:1005A000D72A8630AC008F30AD008E30AE002708E1
:0805B000C4000A30C5006C28EC
:1006000005108510F6302302C600F6302202C7001E
:10061000F6302102C800F6302002C900051503108B
:10062000460C0510031805140000000000004707E1
:1006300085140310C70DC70D8510C707470C0000B0
:1006400005100318051448070310C80DC80DC80D80
:10065000851448070310C80D851048070310C8000B
:10066000C80C0510031805147D304918C807000090
:10067000851400000000000085100830CB00C80C75
:10068000851000000000051003180514000000008C
:100690008514CB0B3F2B8510000000000510261B96
:1006A0000514000000008514000000008510000003
:1006B0000000051038180514000000008514000023
:1006C0000000851000000000000000000510B818B0
:1006D00005140000000085140000000085100000D3
:1006E0000000000000000514000000008514000058
:1006F0000000851000000000000000000510000050
:1007000000008514000000008510000000000510A6
:10071000051105148514000000008501A12986013A
:0A0720000715870185016300932B84
:100800000A2C172C242C312C3E2C4B2C582C652CCC
:10081000722C7F2C8130B000DF30B1000130AC0091
:100820009830AD003030AE00B830AF007828E730F7
:10083000B000DF30B100A130AC00A030AD003030EE
:10084000AE00E330AF0078289230B000DF30B10066
:100850008130AC00E330AD008530AE00A030AF0099
:100860007828C230B000DF30B1003030AC009830B2
:10087000AD00E330AE00C830AF007828E430B000FF
:10088000DF30B100C830AC008630AD003030AE0093
:10089000FF30AF007828C830B000DF30B100213021
:1008A000AC00B830AD00FE30AE009D30AF0078280F
:1008B0008830B000DF30B1009830AC00E330AD00DC
:1008C0008530AE002130AF007828E130B000DF3055
:1008D000B1009930AC00E730AD002130AE00FF3000
:1008E000AF0078288030B000DF30B1008530AC0038
:1008F0000130AD009830AE00FF30AF007828C03036
:10090000B000DF30B100A130AC00A030AD00A430A9
:10091000AE009930AF0078280310280CA90003100E
:10092000A90C0310A90C2908A324AC00A90A2908C2
:10093000A324AD00A90A2908A324AE00A90A290806
:10094000A324AF0002288A010A158207FE34FE3470
:10095000FE34FF34FF34FF34FF347434A034873462
:10096000983498348634FF3498349934A034B034B1
:10097000C834FF348E349C34FF34983421348134AD
:1009800099349D349D3498340534FF34FF34FF345A
:02099000FF3432
:100A000007142C088600071607122D088600871683
:100A100087122E088600071707132F0886008717EE
:100A200087130E280710FF302C06860007160712C2
:100A3000FF302D06860087168712FF302E068600AF
:100A400007170713FF302F06860087178713112813
:100A500087143008860007160712310886008716AB
:100A60008712320886000717071333088600871796
:100A7000871317288710FF303006860007160712E5
:100A8000FF303106860087168712FF303206860057
:100A900007170713FF3033068600871787131A28B6
:100AA0003908A9003F307F25B90E2008A900003081
:100AB00039077F252108A900013039077F25220841
:100AC000A900023039077F252308A9000330390720
:100AD0007F252408A900043039077F252508A900AF
:100AE000053039077F252608A900063039077F25FC
:100AF000AA30A900073039077F25B90E7C280317D3
:100B000083128D0029088C0083168C130C15553028
:100B10008D00AA308D008C14A9018C188D2D0C111C
:060B20008312031308001C
:02400E003F3D34
:024010000000AE
:00000001FF
